:030000000219FDE5
:03000B000200A848
:03002B000201854A
:03005B0002033667
:0300730002032362
:1000800002030406080C10182030406080040608A3
:100090000C10182030406080A0C00003070F1F051F
:1000A000050D050305030302C2AF306308C2638573
:1000B000798AD2AF32C0D0C0E0206221E525601637
:1000C000E473E525F4C3334009758A00D263F579FA
:1000D00001D4F58AD262D0E0D0D0D2AF32C3E526C7
:1000E000334009758A00D263F57901EEF58AC26260
:1000F000E526F4602F30682520720DD0E0D0D0C204
:1001000092C296C294D2AF32C292C296C294206F6B
:100110000C2065097410D5E0FDE57B4290D0E0D05D
:10012000D0D2AF32758A00D263757900C28DD262A7
:10013000211D01C2306805206502D29201C23068DB
:1001400005206502D29401C2306805206502D2966E
:1001500001C2C29330680A2065077411D5E0FDD250
:100160009201C2C29530680A2065077411D5E0FD7E
:10017000D29401C2C29730680A2065077411D5E095
:10018000FDD29601C2C2AFC2AD53E6EFC0D0C0E00F
:10019000D2D3D2AFE57A6009E57760057577004183
:1001A000D0757701C2CEE52A600720744F152A2149
:1001B000FC7800790020742EE580307E01F430E573
:1001C0000278FF53DACF207E0343DA20307E0343E8
:1001D000DA10C2D8C271E580307E01F430E50279D0
:1001E000FFC3E89970CB306103752A18207403753A
:1001F0002A18885CD270E86003755F0020740DE5F2
:100200002B6004152B410C43DA01C2D82070024147
:100210007FA85C206102C270207431C3E894F04072
:100220000374F0F8E8C4540F28F87984B703024146
:100230004CC313C3138721200802C313200A06C32B
:10024000C898F8414C28F8500374FFF8C3E8956546
:100250005003E565F88822E52D54066022206B1FC7
:10026000E536C333C333F8E564C313C313F9C39549
:100270002240028922E82522F52250037522FF85BB
:100280002224A824C3E52495614002A8618825E5BD
:1002900066700241C3C3E8AA669A5003E8FAE4F91B
:1002A000EAC333FBE568F45B29400D2567F8E56791
:1002B00060021567400B41C30AC3E5679A50020507
:1002C0006778FF8826C26FC3E52694F84002D26F94
:1002D00020CF0AD0E0D0D043E610D2AD32C2CF0555
:1002E0003AE57A6009E578600575780061197578F6
:1002F000017801E52A6005307402152AC3E55C9493
:10030000014005755F006119756000756900E55F62
:100310002401F55F5003755FFFD0E0D0D043E610B5
:10032000D2AD32C2AF53E67F7592FA7593FFC260C9
:10033000759104D2AF32C2AF53E6EFC2ADC0D0C0A8
:10034000E0C0F0D2D3D2AFA8FBA9FCE57A6007C326
:10035000E913F9E813F8C2D830710261A853DACF73
:10036000207E0343DA10307E0343DA20D271E58029
:10037000307E01F420E502617F88278928A1D553CA
:10038000DACF207E0343DA20307E0343DA10C2D86E
:10039000C271307402A1C17800E580307E01F43072
:1003A000E502A1C1885CA1A953DACF207E0343DA1C
:1003B00020307E0343DA10C271206102818153DA5A
:1003C000CF207E0343DA10307E0343DA20C2D8D236
:1003D0007188578958C3E89555F8E99556F97B0017
:1003E0007E087A00C3E8948CE994005005755B00A0
:1003F0008173882178A2E6A8216055C3E894C8E9F2
:1004000094005008E4D2E4FB7A0A814EC3E8946871
:10041000E994015008E4D2E3FB7A0F814EC3E894DB
:10042000D0E994025008E4D2E2FB7A1E814EC3E880
:1004300094A0E994055008E4D2E1FB7A3C814EC3D4
:10044000E89498E994085008E4D2E0FB7A787E00BA
:10045000C3E89559FCE9955AFD30E70AECF424010C
:10046000FCEDF43400FD755B00C3EC9AED9E500387
:0F047000755B018859895A85575585585678020A
:10047F00A1A9C3E89527F8E99528F9307C02A18D49
:10048F00307B02A18D307A02A18620750281A4E90A
:10049F00FDE8FC81C3E9C313F9E813F8307902A131
:1004AF0086E9C313F9E813F8307802A186E9C3137C
:1004BF00FDE813FC20612CC3EC941CED9402400268
:1004CF0081DAED701EC3EC94C850180529E5297028
:1004DF00021529C3E529940A5002A1C1755C00D207
:1004EF0070A1C1E529600215297888E6F97400200A
:1004FF007F087896B90302789EE624FAFEE434006A
:10050F00FFC3EC9EFCED9FFD9208B90310A20850AB
:10051F0007207609D276A12C307602C276A2085037
:10052F0016B9030DECF42401FCEDF43400FD0205C3
:10053F004678007900A18DB90315EC33FCED33FD3E
:10054F00C3EC940AFCED9400FD50047C007D00C3C5
:10055F00EC94FFED9400400678FF7900A18DEC85B7
:10056F0072F0A4C5F0A2F733F8790040030205A991
:10057F0078FF79000205A9E9C313F9E813F8307C75
:10058F000EE9600278FFC3E81338F8E43400F9C3CA
:10059F00E894FFE99400400278FF885CD2702061F4
:1005AF0002A1C1741FF4552F4BF52FC274EB7002CB
:1005BF00D274752A18307403752A0A306102A1D5D6
:1005CF0020740353DAFE207403752B06D0F0D0E0AD
:1005DF00D0D0D2AD43E6103279010206057903027D
:1005EF000605790A020605791E02060579640206D8
:1005FF000579C80206057817E4D5E0FDD8FAD9F6D3
:10060F00227A147B7802062C7A107B8C02062C7AC5
:10061F000D7BB402062C7A0B7BC802062CE573D532
:10062F00E001227902E4C295D5E0FDD294D5E0FD38
:10063F00C294D5E0FDD295D5E0FDE920E002D2923B
:10064F0030E002D296E573D5E0FDE920E002C292D8
:10065F0030E002C2967496D5E0FDD9C9EAF8D5E02C
:10066F00FDD8FBDBB8C29522C37C007D0075F0007E
:10067F0005F0EA33FAEB33FB50F6EB13FBEA13FA10
:10068F00C3E9FFE8FEE89AF8E99BF95004EFF9EEA9
:10069F00F8B3EC33FCED33FDD5F0DFEDF9ECF822D8
:1006AF00E889F08A20D2D4F8A9F07B0030F70B7BD1
:1006BF00FFF42401F8E9F43400F9E88520F0A4AD43
:1006CF00F0F8E98520F0A4AFF0FEED2EF974003FAD
:1006DF00FA7C04C3EA13FAE913F9E813F8DCF48B94
:1006EF00F030F70AE8F42401F8E9F43400F9E88966
:1006FF00F0C2D4F8A9F02222C3E54113F9E5401363
:10070F00F8C3E54498F8E54599F9500CC3E894808F
:10071F00E994FF401602073EC3E8947FE994005026
:10072F000302073E787F790002073E788079FF88C1
:10073F0049894A22E5492546F8E54A3547F9854A68
:10074F0020E4300701F43548FA30E709C3EA94F0A2
:10075F00401502077CC3EA940F500302077C78FF11
:10076F0079FF7A0F02077C780079007AF0C3E524CD
:10077F009561500AC374019524500B02079AE54AFC
:10078F0020E70E02079AE54A30E706884689478A2E
:10079F00482278A5E6FAC3E54933F8E54A33F9D19B
:1007AF00AFE930E70BC3E89480E994FF4013E1D43D
:1007BF00C3E8947FE994005002E1D4787F7900E197
:1007CF00D4788079FFE820E715C3E52398F840092E
:1007DF00C3E8940140030207FB78010207FBE8F42A
:1007EF0024012523F840030207FB78FF884B22786A
:1007FF00A6E6FAA847A9481206AFE930E70CC3E806
:10080F009401E994FF4016020830C3E894FFE9947D
:10081F0000500302083078FF790002083078017920
:10082F00FFE920E715C3E54B98F84009C3E89401A9
:10083F0040030208577801020857E8F42401254BBA
:10084F00F8400302085778FF88242278FF20692890
:10085F0079A1E76023E541601F74FF8541F084852E
:0E086F0039F0306A0375F005A4F8C5F0600298
:10087D0078FFC3E895645002A864886322C3E540FD
:10088D0094C8E5419400E563500314019B04600294
:10089D00F563220208A32275E890227883E6FF30E3
:1008AD00EDF9A8BDA9BE0570C3E570940840527559
:1008BD007000E9FA79A0E76044EA7007E571601B02
:1008CD000208DCC3E895716010E5715006600C14E8
:1008DD000208E80460F90208E8E571F571C3947245
:1008ED00401B7561C0C394044013756180C39404AB
:1008FD00400B756140C39404400375610075BB08DE
:10090D0022E561F460020561E570B4070375BB1063
:10091D0022743279A787F0A4C5F0A2F733F8C3E8A3
:10092D0095614002A86188228824882588268864DC
:10093D00227540007541F022C2AF75C820A8CCA920
:10094D00CDAA3A30CF010A75C824D2AFC3EA13FA43
:10095D00E913F9E813F8AB3BAC3C883B893CC3E8A1
:10096D009BF8E99C20690A547FF9306602416421A5
:10097D00BEAD3D8A3DF9EA9D547FFA600678FF7958
:10098D00FF21A3AE3EAF3F8B3E8C3FA83BA93CC39E
:10099D00E89EF8E99FF9C3E54113FBE54013FAE83A
:1009AD002AF540E93BF54150067540FF7541FF4181
:1009BD000BAA40AB41AC40AD417E047F02C3EB942A
:1009CD0004400D1E1FC3EB94084005206A021E1F34
:1009DD00C3ED13FDEC13FCDEF7C3EA9CFAEB9DFBB4
:1009ED00EF6009C3E913F9E813F8DFF7EA28FAEB2A
:1009FD0039FB8A408B4150067BFF8B408B41C3EB0B
:100A0D0094025002D2663069047F0341367892E633
:100A1D00FFC3E537948240110FC3E53794A0400121
:100A2D000FC3EF940640027F057E02E541C4540FCB
:100A3D00F9E541C454F0F8E540C4540F28F8C3E873
:100A4D009EFAE99400FB4009C3EA9402EB9400502E
:100A5D00047A02E4FB41B0AA40AB41EBC4FEEAC408
:100A6D00540F4EFCC3EA9CFAEB9400FBC3E813C38E
:100A7D0013F8EA28FAEB3400FB8A408B41C3EB9460
:100A8D00024002C2667802EBC4FE7B00EAC4540F3A
:100A9D004EFAC3EA98FA4005C3940250027A0278DE
:100AAD0092E6FF30600241B0855192855293D2603B
:100ABD0043E680C3E49AF8E49BF9C3E833F8E933DD
:100ACD00F93066026143E8FAE9FBD3E913FDE81357
:100ADD00FC88518952C3EF94036038EF20E00DE894
:100AED002CF8E93DF9ECFAEDFB020B0CE828F8E9DE
:100AFD0039F9C3E82402F8E93400F97AFE7BFFC323
:100B0D00EF9403400E8A538B54884D894E8C4F8D34
:100B1D00506177885389548A4D8B4E8C4F8D503050
:100B2D0069127553F07554FF754FF07550FF75517F
:100B3D00F07552FF6177E8FAD3E813FC8851C3EFE3
:100B4D0094036020EF20E007E82CF8ECFA6163E8ED
:100B5D00282402F87AFEC3EF940340088A53884D87
:100B6D008C4F617788538A4D8C4FE568C3335002A3
:100B7D00646BF5683060026181753402D26043E6C2
:100B8D0080E52D5406602DA840A941C3E913F9E86D
:100B9D0013F8306904E92440F9C2AF53E67F75912B
:100BAD0000C3E498F594E499F595759104D26043EA
:100BBD00E680D2AF22D264754300752000306C03FD
:100BCD00752040020BE1D264754300752040306CF6
:100BDD000375200078017901206620E52D5406600B
:100BED0002C2647914E541C313700104F8C394146F
:100BFD0040027814306904781B791BC3E833F8C3BD
:100C0D00E933F9206010E543600C306903D53404F5
:100C1D00D26D819871890543E59BF45440B520024E
:100C2D00818230690908C3E8994001188110206458
:100C3D000A08C3E899400261E18110C264C2AF5352
:100C4D00E67F7591003066127594007595F075917B
:100C5D0004D26043E680D2AF61E1E5417EFFC3334C
:0E0C6D004009C3334005C3334001FEC3E49E7B
:100C7B00759400F595815BC3E5339401500261E1F6
:100C8B0030640261E1D80281968110C26DC2AF530C
:100C9B00E67F759100855394855495759104854D28
:100CAB0092854E93D26043E680D2AFE52D54066019
:100CBB0008206A020533020CD4306D0D206C0A201B
:100CCB006407158115810215A9227800306402781A
:100CDB0001E53775F007A4F9E5F028F5F0E9A2F086
:100CEB0013A2F113A2F213F537C39478500375379F
:100CFB0078C3E53795384008D265C292C296C29444
:100D0B00306002A10B854F92855093D26043E680F1
:100D1B0022207D16C2AF754202C295D29330620279
:100D2B00D296D2AF759F40020F0CC2AF754202C272
:100D3B0095D297306202D292D2AF759F40020F0CC0
:100D4B00307243207D20C2AF754203900163757BE7
:100D5B0020C296C297306204D294A169D295D2AFC9
:100D6B00759F41020F0CC2AF754203900163757BF7
:100D7B0020C292C293306204D294A189D295D2AF91
:100D8B00759F43020F0C207D17C2AF754203900174
:100D9B003EC296306202D294D2AF759F41020F0CC5
:100DAB00C2AF75420390013EC292306202D294D21E
:100DBB00AF759F43020F0C207D16C2AF754204C264
:100DCB0093D297306202D294D2AF759F43020F0C2D
:100DDB00C2AF754204C297D293306202D294D2AFA3
:100DEB00759F41020F0C307243207D20C2AF7542BC
:100DFB0005900152757B08C294C295306204D29261
:100E0B00C10FD293D2AF759F40020F0CC2AF754288
:100E1B0005900174757B80C294C295306204D296A2
:100E2B00C12FD297D2AF759F40020F0C207D17C2F6
:100E3B00AF754205900134C294306202D292D2AFA8
:100E4B00759F40020F0CC2AF754205900148C294CA
:100E5B003062EBD296D2AF759F40020F0C207D16FD
:100E6B00C2AF754206C297D295306202D292D2AF10
:100E7B00759F41020F0CC2AF754206C293D29530DB
:100E8B006202D296D2AF759F43020F0C3072442090
:100E9B007D20C2AF754201900174757B80C292C2F6
:100EAB0093306204D296C1B5D297D2AF759F4302ED
:100EBB000F0CC2AF754201900152757B08C296C2EE
:100ECB0097306205D292020ED6D293D2AF759F4164
:100EDB00020F0C207D17C2AF754201900148C292E0
:100EEB00306202D296D2AF759F43020F0CC2AF7520
:100EFB004201900134C296306202D292D2AF759FFA
:100F0B0041C26522900132757B00C292C296C29497
:100F1B00C293C297C295C26222788076FF0876FF91
:100F2B000876FF0876FF08760308760408760A0829
:100F3B007603087601087601788C76010876FF082F
:100F4B0076FF0876FF0876FF0876FF0876030876AB
:100F5B00FF0876FF0876FF0876250876D00876FA24
:100F6B000876FA0876040876FF08760108760008FA
:100F7B00767A0876FF0876010876010876000876FF
:100F8B0003087600227887E6FFC272BF0302D27293
:100F9B007888E6C394036008C27DE630E102D27D17
:100FAB00C27E7889E630E102D27EC3EF94026008FC
:100FBB00758E01D273020FC8758E00C273227880B2
:100FCB00E6149000809378A5F67881E61490008063
:100FDB009378A6F67886E61490008D9378A7F6782A
:100FEB0086E6F539C394025003753902789CE67591
:100FFB0038FFB402037538A0B4030375388278A3A5
:10100B00E61490009A93F566120F0F22227896E65B
:10101B00FA7897E6FB7888E6B40305C3EB940EFBEE
:10102B00307F047A007BFFC3EB9AFCC3948250029F
:10103B007C827572000572EC8572F0A4C3E5F094A6
:10104B007D40F222D27F11181205F61205F67A00B6
:10105B007B007C101205ECE55C2AFA74003BFBDC90
:0F106B00F37C04C3EB13FBEA13FADCF7FEC27F3E
:10107A00111822757C00757D00E5EF20E6037520C6
:10108A00000520903FFFE520146006901FFF1460C2
:10109A00009304600375EF1653D9BF7581C043FFEF
:1010AA00801205E775EF0643B203E5B3240220E791
:1010BA000DF521E5E320E0068521B343E301120F94
:1010CA000F7580FF75A40075F13075D4DF75900334
:1010DA0075A5FC75F2FC75D50175A60175E241127C
:1010EA000F0FE4F8F6D8FD756801120F24121603E3
:1010FA0078988673753001C2AF1206001206101274
:10110A0005F61206171205F612061E1205F6121732
:10111A002C1206001206001205FBC2AF757C007580
:10112A007D0078FA79FA308507D9FBD8F7021C00D6
:10113A00120F90120FC91117111878988673120F8F
:10114A000F75A90075B680757A00758810758902C1
:10115A0075C82475910475D84075A82275B80275AA
:10116A00E690759B80759D0075D10E75BCC075BBE8
:10117A000875BA1175E8801205E7D2AF1208A07592
:10118A00360053DACF207E0343DA20307E0343DA77
:10119A001043DA01C2D8C271120600D2617B037A07
:1011AA000CE55B70077A0CDB030211241205F620AA
:1011BA007003021124C270E55CC3940240E1E52F7A
:1011CA00541F855E5DF55EB55DD5DAD5C26153DA29
:1011DA00CF207E0343DA20307E0343DA10C2D8C21E
:1011EA007178A2E67008D274E52F54E0F52FC27523
:1011FA007529001205FB307409C3E529940A4002D7
:10120A00D2751205EC78023074027800C3E55C9856
:10121A0040F0C2AF120610120610120610D2AF1218
:10122A000600754C007888E6B4030261241205ECC6
:10123A00788CE6C394015003021324E530C3940169
:10124A005003021324757CA5757DF1207435C3E51E
:10125A005C94FF5003021324C2AF120625D2AF12C8
:10126A0005FBC3E55C940150EFC2AF1206101205EC
:10127A00F1120610D2AF1205FBC3E55C94FF40E9F8
:10128A000217B17F05D27F11181205FBC2AFC27FC8
:10129A001118AE5CC3E55C947FD2AF500261341280
:1012AA0005E7C2AF120625D2AFDFDA114FC3EE94BB
:1012BA00057897F61206001217347F0AD27F1118A2
:1012CA001205FBC2AFC27F1118AE5CC3E55C947F06
:1012DA00D2AF50E61205E7C2AF1206101205F1129C
:1012EA000610D2AFDFD6114FEE24037896F6F879BE
:1012FA0097E7C394824003985006E824827897F6C9
:10130A001206001216511217631205FB1118C3E5D3
:10131A005C94FF5002414F0217B1757C00757D0045
:10132A00C3E55C954C4003855C4C1205FB7801795A
:10133A0088E7B403027805C3E55C984002412FC2EE
:10134A00AF120625120625120625D2AF120600751F
:10135A003000E4F531F5320531E531F4703F0532FC
:10136A00789AE67819146012783214600D787D1430
:10137A00600878FA146003753200C3E53298401D9C
:10138A00120F0F1205E7153275310078998673C26C
:10139A00AF120625D2AF789886731205FB1205F1B3
:1013AA00E52A700530740221247801207402780637
:1013BA00C3E55C9840A17888E6C3940360031205EC
:1013CA00FBE52A7003021124C2AF120F0FE4F522C3
:1013DA00F523F524F525F526F567D2AF7885E6C31A
:1013EA0033F565E4F544F545F546F547F548F570F6
:1013FA00F52CF52DF53775700875BB101205E71237
:10140A0008A430EDFDA8BDA9BEE97001F8887112E3
:10141A0008A875700875BB10120F90C2AF7561FFEE
:10142A0012091E852261852262852263D2AF752246
:10143A0001752401752501752601856069756A01A2
:10144A0075B69075A903757A017888E6B40307C260
:10145A007D307602D27DD268D269753300120E6869
:0F146A00120E9712093E12094512093E1209454A
:1014790012093E120BD3120706120CD5120D1C12BB
:101489000945120BC2306E031207072066031208C2
:101499005A30660312088A120CD5120D4B120945EF
:1014A900120BD3306E03120743120CD5120DC21260
:1014B9000945120BC2306E031207A1120CD5120D89
:1014C900F1120945120BD3306E031207FE120CD527
:1014D900120E681209451208A4120BC2120CD51279
:1014E9000E971208A812094530692F856461856431
:1014F90062856069756A0179187A0CC3E533994088
:101509000CC269D26A8A357561FF021523C3E55C8D
:101519009401400302147C0215B1306A25206C2223
:10152900E535147006C26AD26B817CF535C3E55C7A
:101539009401400302147C7888E6C3940360030293
:1015490015B1753600788279A4E760027803C3E59E
:101559005F985054307404E52A604D7888E6B403E6
:1015690017207D05207607A181307602A181206CA4
:1015790007D26C85646181BB78F0306C0585646144
:101589007820C3E541985002817C306C1BC26CC243
:101599007D307602D27DD26A753512856461817C8F
:1015A9000536E55C6002A1B4753600C2AF120F0FB3
:1015B9007887E6FE7602120F907887EEF6E4F52238
:1015C900F523F524F525F526F565752C00752D000F
:1015D90075A90075B680757A00D2AF1205FB120F96
:1015E9000F78A4E66006D293D295D297307409C3D6
:1015F900E536940440022124615C901A0D7820128A
:101609001693E520B45A0CA3121693E520B4A5034A
:10161900021631757CA5757DF1120F2412165175CC
:101629007C00757D00021650901A0378807B0A129F
:101639001693A308DBF9901A0F788C7B191216936D
:10164900A308DBF9901A2822C2AF1216D61216B3D4
:10165900901A00740E121698A37409121698A3749E
:1016690015121698901A0378807B0A121697A30808
:10167900DBF9901A0F788C7B19121697A308DBF9FE
:101689001216E91216C7901A2822E493F622E643A5
:101699008F01538FFDFFC3E583941C400122EF8521
:1016A9007CB7857DB7F0538FFE22438F02438F01AC
:1016B900857CB7857DB7901A0DF0538FFC22901A5F
:1016C9000D745AD198901A0E74A5D198227A30794E
:1016D900D07820901A40D193E520F709A3DAF722B0
:1016E9007A3079D0901A40E7D19809A3DAF922AB78
:1016F90074A875BB01027984BB02027985BB030218
:101709007986BB04027992BB05027987BB06027907
:10171900A3BB0702799CBB08027988BB09027989B6
:10172900E8F7227C05120600DCFB22C2AF12061084
:1017390012061712061E1206251205F112061012BC
:10174900061712061E1206251205F11206101206B8
:101759001712061E120625D2AF22C2AF1206251293
:10176900061E1206171206101205F1120625120698
:101779001E1206171206101205F112062512061E70
:10178900120617120610D2AF22AE74AF75C2AF128D
:1017990006101206101206101205F1DEF2120625C5
:1017A9001205F1DFF8D2AF22F134F12CF12C757466
:1017B90001757501757600F1927C05AD5C12060024
:1017C900C3ED955C70F5C3E55C9401400AC3E55C23
:1017D90094FF40320217EDD1F8D151F134C2AF75FF
:1017E900EF16F12CDCD50576C3E57694035002801B
:1017F900C6F12C0575E5741490009F93F808C3E5AC
:101809007598500280AE12172C12172C0574C3E577
:1018190074940A5002809A120F24121651C2AF759D
:05182900EF1612172C60
:0319FD0002107D58
:101A00000E0915FFFFFFFF03040A0301015AA50198
:101A1000FFFFFFFFFF03FFFFFF25D0FAFA04FF01DE
:091A2000007AFF0101000300FF40
:101A4000234459535F584D32304123202020202019
:101A500023424C48454C492346333930232020202B
:101A60002020202020202020202020202020202076
:101C0000C2AFC2D353D9BF7581C043B20343FF8073
:101C1000752438752503B1DC7529A5752AF175E29F
:101C20004043F12053A4DF75D4FFD2857DFA7803B9
:101C300079E67C10752200752300901DE97B0675FE
:101C400024987525013085028145208508D8FBD967
:101C5000F9DCF781B7308508D8FBD9F9DCF781B713
:101C6000B19CE493A3C39A6004DDC381B7DBDBB10D
:101C70008E6002812E7B08E493FAA3B16FDBF87AC1
:101C800030B16F752200752300B18EEAFCEBFDC305
:101C9000ED94FE400EB18E8A278B28ED30E0048A49
:101CA000828B83B18E7AC270D8C3ED94FE601950D6
:101CB000CEBD002BEC600F7520007521FF7529004B
:101CC000752A000200008100A827A9280809D80465
:101CD000D90281DCB192EA89AAF281CE0D81A3C337
:101CE000ED94035053EDA2E092007AC5C3E58294CF
:101CF00000E583941C508A200010438F02438F011B
:101D00008529B7852AB7F0300029A827A92808090E
:101D1000438F01538FFDD804D902A133C3E58394C7
:101D20001C4003A3A11689AAE28529B7852AB7F02A
:101D3000A3A116538FFC817F7AC1BD030CE493A34A
:101D4000FAB153DCF8B14B817F8181AA22AB23B178
:101D50006FEBFAEA6222752608C3E52313F523E543
:101D60002213F52250066323A0632201D526EAB18F
:101D7000DCB1DC75260AEAF4200102D285300102CA
:101D8000C285B1DCC3134002C201D526EB22B19259
:101D9000EAFB208502A192308502A197752608AE44
:101DA00024AF25C3EF13FFEE13FEB1E0B1DCC3EAAD
:101DB000133085024480FA30E703632201C3E52330
:101DC00013F523E52213F52250066323A0632201B5
:101DD000D526D9E52265236523F52222AE24AF2539
:101DE0000E0FDEFEDFFCD20122424C48656C6934E6
:071DF000373164F390060196
:00000001FF
